:103BCC00C2AF53FFBFE4F5F18EF38FF212000AAFD0
:063BDC00F443FF40D2AFEC
:013BE20022C0
:103B9700C2AF53FFBF75F1A08EF38FF2AF058FF45D
:0B3BA70012000A43FF40D2AFAFF4222F
:1039D0009062AEEEF0A3EFF0C2AF53FFBF75F1807F
:1039E00012000A75F1309062AEE0FEA3E0FF8EF3A4
:0E39F0008FF2E4F5F412000A43FF40D2AF223A
:01000A0022D3
:103C5000EEF0A3EFF0E4A3F0A3F022E0FEA3E0FF78
:023C6000C3227D
:1038DC009061FD123C509061FD123C5B906200E0E7
:1038EC009F9061FFE09E501A000000000000000055
:1038FC000000906200E004F070DC9061FFE004F0E6
:03390C0080D42242
:103941009061F9123C509061F9123C5B9061FCE08E
:103951009F9061FBE09E50177FE87E031238DC9058
:1039610061FCE004F070DF9061FBE004F080D7229D
:103971009062A6123C509062A6123C5B9062A9E054
:103981009F9062A8E09E50177F0A7E0012394190F5
:1039910062A9E004F070DF9062A8E004F080D72211
:103C6200759850438920438780758BFC758DFCD2F3
:023C72008E22A0
:073CB800C298C299D2AC22B0
:083CB0008F993099FDC29922A1
:1027A200F090627EE03400F0906274E0FF90626E1E
:1027B200E0FBA3E0FAA3E0F9EF12140A906275E0DD
:1027C20090626EFFE0FBA3E0FAA3E0F92290620BB5
:1027D200E0FEE42401FFEE3440FE22EFF0A3EBF032
:1027E200A3EAF0A3E9F022906268E0FF90627EE043
:1027F200FCA3E0AA04F97B00220B906219EBF0A380
:102802007462F0A37474F0A3E4F0A322FEE4241132
:10281200FFEE3440FEA3E0FD22900001EF12141CF3
:10282200906276E090000212141C906277E09000B1
:102832000312141C906278E02290620BE0FEE42402
:1028420024FFEE3440FE2290620BE0FEE42425FFDA
:10285200EE3440FE22EFFD7C00E0FEE42DFFEC3E74
:102862002290620BE0FEE42428FFEE3440FE229028
:10287200620BE0FEE42429FFEE3440FE22E4F0A3E2
:10288200F0A3F0A3F02225E0249BF582E43461F565
:1028920083E022E0FF90627CE4F0A3EFF0E0FE220E
:1028A200906279E07C002400FFEC3E22900003025B
:1028B20013DD90620BE0FEE42404FFEE3440FE22BE
:1028C200FFEE3440FE90628622FFEE3440FEA322E9
:1028D200E0FDA3E090621ECDF0A3EDF022E0FDA3A7
:1028E200E090621CCDF0A3EDF022FEF0FCA3EFF02D
:1028F200FD22E0F9A3E0FAA3E0906219C922E0FE0A
:10290200E42400FFEE3440FE22E0FFAA04A9059071
:10291200621BE4229000010213DD9000020213DD2B
:1032490090620BEFF090620DEAF0A3EBF090620C44
:02325900EDF096
:10325B0064016018E0FF64026012EF6403600DEF1D
:10326B0064046008EF6405600302330490620BE0B2
:10327B00FF123B1690620B12290090620FE0FD903B
:10328B00620CE04DFD123C1190620DE0FCA3E04C92
:10329B00601C1228B4C006C007ECFDD007D0061284
:1032AB00330F2405FFEE3440FE90620D802C9062AC
:1032BB00B1E004F070069062B0E004F01228B4C0E4
:1032CB0006C0079062B0E0A3FDD007D00612330F03
:1032DB002405FFEE3440FE9062B0A3E0FD123C11DA
:1032EB001227CF7D01123C111227CF123B46EF70F4
:1032FB00F79062107401F08005E4906210F0906218
:03330B0010E0FFD0
:0B330E0022123C1190620BE0FEE42252
:103B1600906217EFF01227D37D10123C11906217B6
:103B26001227D2123B46EF70F4906217E0FF7DFF3A
:033B3600023C85C9
:05386F0090620BEFF078
:10387400123C26EF6413701F90620B1227D27D0254
:10388400123C1190620B1227D2123B46EF70F49057
:10389400620C7401F08005E490620CF090620CE01C
:0138A400FF24
:0138A5002200
:062CFC009062981227DD32
:102D02001213C4FFB4FF189062991227C612291633
:102D1200B4FF0C12291CB4FF061228AEF46022EF95
:102D220070159062991227C6122916700A12291C70
:102D320070051228AE600A90629CE07002A3E070F7
:102D420008E490629EF0022DFA90629E7401F09067
:102D52006298E0FEE4240C1228CB1227C61213C498
:102D6200122E0E240D1228CB1227C6900001122E0D
:102D720000240E1228CB1227C6900002122E002425
:102D82000F1228CB1227C61228AE122E0E2410FFC5
:102D9200EE3440FEC006C00790629CE0A3FDD0075F
:102DA200D006123C11906298E090629C12280E129A
:102DB2003C11123A579062981227D27D04123C11AC
:102DC2009062981227D2123B46EF70F4122E1964C9
:102DD200156022122E196417601B906298E0FF1290
:102DE2003CA7EF30E3E6906298E0FF7D08123C8555
:0D2DF200E490629EF0123BFA90629EE0FFBA
:102DFF00221213DDFD123C11906298E0FEE422FDD9
:102E0F00123C11906298E0FEE422906298E0FEE49A
:0C2E1F002403FFEE3440FE123B46EF227D
:103BB20090620BEFF01227D37D08123C1190620B3A
:0A3BC2001227D2123B46EF70F422E6
:062BC20090620B1227DDFA
:102BC80090621112287FA3F0A3F090620BE0FE122E
:102BD8002888FCA3E0FD90620FE0FAA3E0FBD39DF8
:102BE800EA9C4011EE122888FDA3E0906215CDF012
:102BF800A3EDF08008906215EAF0A3EBF090620B69
:102C0800E0FF1236B8906213EEF0A3EFF0122CF248
:102C18006417600EEF641C6009E4906215F0A3F07D
:102C28008015906215E0FCA3E0FDC3906214E09D5E
:102C3800906213E09C40C612283B123B46906211FA
:102C4800E4F0A3EFF0122849123B469062121228D2
:102C5800579062111228EC90620B12290B1227E18F
:102C68009062151228D290620C1227C61230619019
:102C78006215E0FEA3E0FF906212E02FF09062116F
:102C8800E03EF012283BC006C007906211E0A3FDA9
:102C9800D007D006123C11122849906211A3E0FD1A
:102CA800123C1190620B1227D27D20123C119062C7
:102CB8000B1227D2123B46EF70F490620BE0FF1222
:102CC8003CA7EF20E411122CF270EF90620BE0FFAA
:102CD800123B16E4FEFF2290620BE0FF7D10123CCF
:092CE80085906215E0FEA3E0FFF7
:0B2CF1002290620BE0FF123C26EF2255
:0633190090620B1227DD9B
:10331F0090621112287FD3906210E0940090620F98
:10332F00E0940050030233D4122863123B4690629C
:10333F0011E4F0A3EFF0122871123B4690621212C3
:10334F0028579062111228EC90620BE0FFAA04A993
:10335F00057B00C002C001A31228F41227E190627E
:10336F000F1228DFD001D00212316090620FE0FE01
:10337F00A3E0FF906212E02FF0906211E03EF01296
:10338F002863C006C007906211E0A3FDD007D006E6
:10339F00123C11122871906211A3E0FD123C1190A2
:1033AF00620B1227D27D40123C1190620B1227D272
:1033BF00123B46EF70F490620FE0FFA3E0906213B0
:0D33CF00CFF0A3EFF0906213E0FEA3E0FF4B
:0133DC0022CE
:062463009062801227DDEB
:10246900E490628B122880906280E0122888FEA393
:10247900E0FF906284E0FCA3E0FDD39FEC9E9062B4
:102489008B4007EEF0A3EFF08005ECF0A3EDF090A0
:1024990062861227C61213C4700F122916700A1207
:1024A900291C70051228AE6014906289E07002A39D
:1024B900E0600A90628BE07002A3E0700AE4906227
:1024C9008BF0A3F00225DD906280E0FEE4240CFF8E
:1024D900EE3440FE1213C41225F4240D1228C21240
:1024E90027C69000011225E6240E1228C21227C61B
:1024F9009000021225E6240F1228C21227C61228BC
:10250900AE1225F42410FFEE3440FEC006C0079039
:102519006289E0A3FDD007D00612260BE0906289FC
:1025290012280E12260B12283E123B4690628DE4A9
:10253900F0A3EFF090628012284C123B46EFFD7C2D
:102549000090628E12285BFE90628D1228ED9062D7
:102559008012290B1227E190628B1228D290628196
:102569001227C612306190628BE0FEA3E0FF9062F1
:102579008EE02FF090628DE03EF090628012283E4E
:10258900C006C00790628DE0A3FDD007D006123CBB
:102599001190628012284C90628DA3E0FD123C11CB
:1025A900123A579062801227D27D20123C11906214
:1025B900801227D2123B46EF70F412261220E40F44
:1025C90012261230E3F47D181225FFE4FEFF227D66
:0C25D900101225FF90628BE0FEA3E0FFD3
:1025E500221213DDFD123C11906280E0FEE422FD13
:1025F500123C11906280E0FEE422906280E0FF12BE
:102605003C85123BFA22123C119062802290628036
:07261500E0FF123CA7EF22D9
:06261C009062681227DD48
:10262200E490627C122880D390626DE09400906204
:102632006CE094005003022791906268122866129F
:102642003B4690627EE4F0A3EFF090626812287439
:10265200123B46EFFD7C0090627F12285B90627E07
:10266200F0A3EFF0906268122900123B46EF540784
:1026720024FD60531460732402600302277A122738
:10268200E9C0031227FB7408F0D00312279A24082A
:102692001227A212281B9062711227C5E48FF01232
:1026A20014B79062711227C6121454FE1228A28F18
:1026B200F01214B790627A12289590627BE024009F
:1026C200FFEC3EA302271F1227E9C0031227FB7467
:1026D20006F0D00312279A24061227A212281B12F0
:1026E20028961228A290627C80331227E9C0031236
:1026F20027FB7402F0D00312316090627FE0240263
:10270200F090627EE03400F090627412289590623C
:10271200751228A5CF24FECF34FF90627CF0A3EF80
:10272200F01227E9C002C0019062691228F4122750
:10273200E190627C1228DFD001D0021231609062F7
:102742007CE0FEA3E0FF90627FE02FF090627EE0EB
:102752003EF0906268122866C006C00790627EE072
:10276200A3FDD007D006123C119062681228749023
:10277200627EA3E0FD123C119062681227D27D4076
:10278200123C119062681227D2123B46EF70F4900D
:07279200627CE0FEA3E0FF02
:092799002212316090627FE022FF
:102F4C003D3D3D3D3D3D3D3D3D3D3D3D3D3D3D3DA5
:102F5C003D3D3D3D3D3D3D3D3D3D3D3D3D3D3D3D95
:102F6C003D3D3D3D3D3D3D3D3D3D3D3D3D3D0D0AE8
:102F7C0000202020202020205737313030412020C5
:102F8C004E657420436F6E66696720496E666F727A
:102F9C006D6174696F6E2020202020202020200D70
:102FAC000A004D414320414444524553532049505B
:102FBC00203A20252E3262782E252E3262782E254C
:102FCC002E3262782E252E3262782E252E326278A1
:102FDC002E252E3262780D0A00252E3362752E2591
:102FEC002E3362752E252E3362752E252E33627587
:102FFC00005355424E4554204D41534B20203A200E
:10300C0025730D0A00472F57204950204144445244
:10301C00455353203A2025730D0A004C4F43414C25
:10302C002049502041444452455353203A202573A3
:10303C000D0A00C0A80102C0A80101FFFFFF00009B
:10304C0008DC112233020202020202020202020214
:05305C00020202020265
:0B3B7A004861AB0000000000000000EC
:10292200906200E025E0FF9061FFE033FE749B2F90
:10293200F58274613EF58322906200E025E0FF900B
:1029420061FFE033FE748B2FF58274613EF58322C2
:10295200AC02AD03C39DFFEE9CF0A3EFF0A3E0FE3B
:10296200A3E0FFE422F0A3E4F0747B2FF58274610C
:102972003EF58322F0A3E4F0746B2FF58274613E7E
:10298200F58322FFEE3440FEE0FBA3E0FAA3E0F978
:102992008D828C831213DDFD123C119061FFE0FCED
:1029A200A3E0FD227D017BFF7E007F0402139E2FA8
:1029B200FFE43EFEED34FEFDEC338F0F8E0E8D0DE7
:1029C200F50C2225E024B7F582E43461F583E0FEBC
:1029D200A3E0222FFFE43EFEE434FEFDE433FC22BA
:1029E2007D017BFF7E007F0802139E7A00AB07E029
:1029F200FEE422E0F510A3E0F51122EFFD7C00EBEE
:102A0200FEE42DFBEC3EFA4B228F0F8E0EF50DF5F8
:102A12000C22F583E05AFEA3E05FFBAA06E922FE40
:102A2200E42DFFEC3EF0A3EFF022F583E0FCA3E0FF
:102A3200C39FEC9E22C2AF7593FE8F828E8322EFDC
:102A4200F0E4A3F0A3F0FBFA2290620BE0FEE42292
:102A5200A3E0FAA3E0FF2225E024C7F582E4346173
:102A62002225E0249BF582E434612225E0248BF5C3
:052A720082E434612242
:103BE300123CC5C2AF123C6275EBFF75ECFF75ED7D
:073BF300FF75EEFFD2AF22C7
:101D660078317C627A30793F1229A678357C627A9E
:101D76003079431229A678397C627D017BFF7A305F
:101D860079471229AA783D7C627D017BFF7A3079FA
:101D96004B7E007F0612139E78437C627A3079511F
:101DA6001229E2784B7C627A3079591229E27B015A
:101DB6007A627939123A819062317F0F121FAE90A2
:101DC60062327F10121FAE9062337F11121FB690DF
:101DD60062347F12121FB69062357F01121FBE90C9
:101DE60062367F02121FBE9062377F03121FC690B3
:101DF60062387F04121FC6123BFA90623D7F0912B9
:101E06001FCE90623E7F0A121FCE90623F7F0B125A
:101E16001FD69062407F0C121FD6906241E0FD7F74
:101E26000D7E00123C11906242E0FD7F0E7E001294
:101E36003C119061FC7401F0A37462F0A3744BF042
:101E46007B017A62794312224C121FEC7BFF7A2FB8
:101E5600797D121A6C121FEC7F097E00123B46C078
:101E6600077F0A7E00123B46C0077F0B7E00123BAF
:101E760046C0077F0C7E00123B46C0077F0D7E00E2
:101E8600123B46C0077F0E7E00123B46906211EF62
:101E9600F0906210D0E0F090620FD0E0F090620E09
:101EA600D0E0F090620DD0E0F090620CD0E0F07BD4
:101EB600FF7A2F79AE121A6C7B017A627964123A34
:101EC600CD90620C74FFF0A3742FF0A374E5F0902C
:101ED6006264E090620FF0906265E0906210F090AC
:101EE6006266E0906211F0906267E0906212F07BA9
:101EF600017A627953121A6690620C7401F0A37427
:101F060062F0A37453F07BFF7A2F79FD121A6C7F6F
:101F1600017E00123B46C0077F027E00123B46C090
:101F2600077F037E00123B46C0077F04121FDED0E8
:101F3600E0F0906210D0E0F090620FD0E0121F85C2
:101F46007A307911121A6C7F0F7E00123B46C00759
:101F56007F107E00123B46C0077F117E00123B4673
:101F6600C0077F12121FDED0E0F0906210D0E0F0C2
:0F1F760090620FD0E0121F857A307927021A6C23
:101F8500F090620C74FFF0A3742FF0A374E5F07B5E
:101F9500017A627953121A6690620C7401F0A37487
:101FA50062F0A37453F07BFF22E0FD7E00123C112A
:101FB50022E0FD7E00123C1122E0FD7E00123C1164
:101FC50022E0FD7E00123C1122E0FD7E00123C1154
:101FD50022E0FD7E00123C11227E00123B469062FB
:101FE50012EFF0906211227BFF7A2F794C121A6C56
:011FF50022C9
:043CC50075FF402225
:103C740075FE0843FE207F647E0012394153FEDF47
:013C8400221D
:103C1100A2AFE433FC122A37EDF0E4F593AF04EFE1
:043C210024FF92AF3B
:013C2500227C
:0D3B3900906217E0FEE42420FFEE3440FE11
:103B4600A2AFE433F9122A37E0FFE4F593AD01EDB5
:043B560024FF92AF07
:013B5A002248
:093CA700EFFEE42402123B41226D
:0D3C8500EFFEE42402FFEE3440FE023C118D
:0B224C009061F9EBF0A3EAF0A3E9F0C9
:10225700E4906201F0A3F0A3F0A3F09061C774804B
:10226700F0A3E4F09061B774C0F0A3E4F09061FFCD
:10227700F0A3F012299DFEE4241F9061F91229852D
:10228700FEE4241E9061FC12298525E0FFEC12294B
:102297002DE4F0A3F0122947E4F0A3F0C390620104
:1022A700E0648094C050679061F9E0FBA3E0FAA373
:1022B700E0F98D828C831213DD24FE601D24FE60FD
:1022C7002624FC602E24F86036240F704112292240
:1022D7007404122967740302231012292274081246
:1022E70029677407022310122922741012296774B0
:1022F7000F80161229227420122967741F800A1270
:1023070029227440122967743FF0A374FFF0C39029
:102317006203E0648094C050729061FCE0FBA3E02C
:10232700FAA3E0F9A3E0FEA3E0FFF5828E83121380
:10233700DD24FE602224FE602B24FC603324F86039
:102347003B240F7046EF25E0FFEE12294574041277
:102357002976740302238D12293A74081229767498
:102367000702238D12293A7410122976740F8016EA
:1023770012293A7420122976741F800A12293A7496
:1023870040122976743FF0A374FFF012299D25E0CF
:10239700FFEC12292DE0FAA3E0FB906202E02BF09C
:1023A700906201E03AF0122947E0FEA3E0FF906255
:1023B70004E02FF0906203E03EF0ED4C607B90610B
:1023C700FFA3E025E0FFEC33FE74992FF5827461DB
:1023D7003EF583E0FAA3E0FB74C52FF58274613EF6
:1023E7001229CE2BFBEE3AFAED25E0FFEC33FE7413
:1023F700C72FF58274613EF583EAF0A3EBF0748989
:102407002FF58274613EF583E0FCA3E0FD74B52FE0
:10241700F58274613E1229CE2DFDEE3CFC906200E0
:10242700E025E0FF9061FFE033FE74B72FF582747B
:10243700613EF583ECF0A3EDF0906200E004F070EC
:10244700069061FFE004F0C3906200E09408906199
:0B245700FFE064809480500302227AB2
:012462002257
:023C2600AC07E9
:103C28007BFFECFEE42403123B41EF6B6004AB071F
:023C380080F01A
:013C3A002267
:0336B80090621706
:1036BB00122A41123B399062171229ED2421123B39
:1036CB00411229FD6022123B39906218E4F0A3EFFE
:1036DB00F0906217E0FEE42421123B41EFFD906273
:1036EB0019E0906218122A21906218E0FEA3E0FF05
:0736FB006B7002EE6A70BC67
:0137020022A4
:0336660090620B64
:10366900122A41122A4B2426123B4190620B12293D
:10367900ED2427123B411229FD6024122A4B2426EE
:10368900123B4190620CE4F0A3EFF0122A4B24277D
:10369900123B41EFFD90620DE090620C122A2190DD
:0E36A900620CE0FEA3E0FF6B7002EE6A70B5EB
:0136B70022F0
:05306100906217EFF082
:10306600AF01906222EAF0A3EFF090621B122A529F
:10307600906217E0F925E0247BF582E43461122A98
:1030860014122A591229CE2BFFEE3A906224F0A38D
:10309600EFF090621FE02BFF90621EE03AFEE9120D
:1030A6002A63122A2C4003023138906217E0122A52
:1030B600631229CE906220122952FCFDC004C0057D
:1030C600C006C00712295F1229B19062201229F5A5
:1030D600D007D006D005D00412354C906220E0FE11
:1030E600A3E0FF906223E02FF0906222E03EF0C35F
:1030F60090621FE09FFF90621EE09E906220F0A308
:10310600EFF0906217E0122A59F583E0FFA3E090F2
:103116006224CFF0A3EFF0906222122960FCFDC07A
:1031260004C005C006C00712295F1229B1906220AB
:103136008019906222122960FCFDC004C005C006F9
:10314600C00712295F1229B190621E1229F5D00715
:09315600D006D005D00412354C5E
:01315F00224D
:0E316000906215EFF0A3EBF0A3EAF0A3E9F004
:10316E00A3122A52906222EAF0A3EFF09062161296
:10317E002A52906215E0F925E0246BF582E4346161
:10318E00122A141229C52BFFEE3A906220F0A3EFFB
:10319E00F090621DE02BFF90621CE03AFEE9122ACD
:1031AE006D122A2C5074906215E0122A6D1229CEDF
:1031BE0090621E1229521229D5C006C00712295F2D
:1031CE00122A0B90621E1229F5D007D00612354C2A
:1031DE0090621EE0FEA3E0FF906223E02FF090626B
:1031EE0022E03EF0C390621DE09FFF90621CE09EC5
:1031FE0090621EF0A3EFF0906215E01229C5FF90C9
:10320E006220EEF0A3EFF0E41229D5C006C007123B
:10321E00295F122A0B90621E80169062201229607E
:10322E001229D5C006C00712295F122A0B90621C04
:0A323E001229F5D007D00612354C16
:013248002263
:103A81001213C49061B3F09000011213DD9061B480
:103A9100F09000021213DD9061B5F0900003121353
:063AA100DD9061B6F02289
:103A57009061B3E0FD7F057E00123C119061B4E0F8
:103A6700FD7F06123C119061B5E0FD7F07123C1106
:0A3A77009061B6E0FD7F08023C11EB
:103BFA00E4FD7F05FE123C117F06123C117F07127D
:073C0A003C117F08023C1190
:103ACD009061B3E012140A9061B4E09000011214F9
:103ADD001C9061B5E090000212141C9061B6E0904C
:053AED00000302141C9F
:10354C008F0B8E0A8D098C08A2AFE433F51485938A
:10355C001578101214E7A907AF0FAE0EAD0DAC0C19
:10356C0078101214E7AB07C2AFE5111511AE10704D
:10357C000215104E60228993780812152A8F828EBC
:10358C0083E0751200F5138B93AA13780C12152A8D
:10359C008F828E83EAF080D1E51424FF92AF8515DB
:0235AC00932268
:102A77000D0A414343455320492F4F2050726F643D
:102A8700756374732C20496E632E0D0A4D6F646550
:102A97006C204554482D44494F2D343820466972DF
:102AA7006D77617265205265766973696F6E20254F
:102AB700782E2578206275696C643A25732040204A
:102AC7002573200D0A0030382F32372F3138003167
:102AD700333A34353A3038004D414320414444526B
:102AE70045535320495020202020203A20252E32BC
:102AF70062782E252E3262782E252E3262782E2588
:102B07002E3262782E252E3262782E252E3262786A
:102B17000D0A00252E3362752E252E3362752E255C
:102B27002E3362752E252E33627520005355424E83
:102B37004554204D41534B20202020202020203A6F
:102B47002025730D0A004761746577617920495024
:102B57002041444452455353203A2025730D0A001F
:102B670049502041444452455353202020202020DF
:102B77002020203A2025730D0A004F505431203D64
:102B87002025632020202020004F505432203D2054
:102B970025630D0A004950204144445245535320B0
:102BA700202020203A2025730D0A00080201010188
:0B2BB700010101080201010101010100
:053B85004200000000F9
:0B3C92007D017BFF7E007F0802139E77
:033CC900C2B7225D
:033CCC00D2B7224A
:1016850078E97C617A2B79B2123C9278F17C617AA7
:101695002B79BA123C92E4902105F0902104F012C6
:1016A5003BE39061FC7401F0A37461F0A374F1F065
:1016B5007B017A6179E912224C75FF28E4F59DF5E5
:1016C5009E759203758E02759C3F1235AE90620C25
:1016D5007401F0A37425F0A374FFF0A3742AF0A39A
:1016E50074CDF0A374FFF0A3742AF0A374D6F07B35
:1016F500FF7A2A7977121A6C7F097E00123B46C061
:10170500077F0A7E00123B46C0077F0B7E00123B17
:1017150046C0077F0C7E00123B46C0077F0D7E004A
:10172500123B46C0077F0E7E00123B46906211EFCA
:10173500F0906210D0E0F090620FD0E0F090620E71
:10174500D0E0F090620DD0E0F090620CD0E0F07B3C
:10175500FF7A2A79DF121A6C7F057E00123B46C09C
:10176500077F067E00123B46C0077F077E00123BBF
:1017750046C0077F081219BAD0E0F0906210D0E099
:10178500F090620FD0E01219447A2B7933121A6C5B
:101795007F017E00123B46C0077F027E00123B465A
:1017A500C0077F037E00123B46C0077F041219BAAB
:1017B500D0E0F0906210D0E0F090620FD0E0121906
:1017C500447A2B794D121A6C7F0F7E00123B46C06E
:1017D500071219D9C0071219E1C0071219AAD0E0DA
:1017E500F0906210D0E0F090620FD0E012196D7A9F
:1017F5002B7967121A6C2089047F0180027F009083
:1018050061D7EFF07A2B79811219E9208B047F01DA
:1018150080027F009061D7EFF07A2B79901219E959
:101825009001027401F07A007B027DE17CCAE4FF3D
:10183500120DB27F011219967F021208007F031262
:1018450019967F041219F57F051219F57F061208FE
:10185500001237C3902103E0602A14F07F017E0057
:10186500123941902103E0701B7B017A41793212D4
:1018750037867B017A4179361237497B017A41797E
:101885003A1238A6308B33902105E0702D123703BC
:101895001219C8C0071219D9C0071219E1C00712D9
:1018A50019AAD0E0F0906210D0E0F090620FD0E07D
:1018B50012196D7A2B799C121A6C208B05E49021F4
:1018C50005F030896C902104E07066123A2B1219EC
:1018D500C8C0077F107E00123B46C0077F117E00FF
:1018E500123B46C0077F127E00123B46906212EF04
:1018F500F0906211D0E0F0906210D0E0F090620FAD
:10190500D0E0F090620C74FFF0A3742BF0A3741A6E
:10191500F07B017A6179D8121A6690620C7401F035
:10192500A37461F0A374D8F07BFF7A2B799C121A0B
:0F1935006C30890302182BE4902104F002182B68
:10194400F090620C74FFF0A3742BF0A3741AF07B74
:10195400017A6179D8121A6690620C7401F0A3744A
:1019640061F0A374D8F07BFF22F090620C74FFF056
:10197400A3742BF0A3741AF07B017A6179D8121A3C
:101984006690620C7401F0A37461F0A374D8F07BC8
:10199400FF227A017B037DE07CCA1208007A017B76
:1019A400037DE07CCA227F127E00123B46906212C5
:1019B400EFF0906211227E00123B46906212EFF02B
:1019C400906211227B017A4179321237867F0F7E31
:1019D40000123B46227F107E00123B46227F117E7E
:1019E40000123B46227BFF243090620CF0121A6CEA
:0D19F400221208007A017B037DE07CCA22EC
:1037C300900000E07002A3E0601A90000074FFF51F
:1037D300F012143EFEC3E5F09440EE6480948050F2
:1037E3001A023CC9900102E06011900000E4F0A3CA
:0B37F3007480F0123CCCE4900102F066
:0137FE0022A8
:03002300023CBFDD
:063CBF00309802C29832A9
:10360C0090620BE0FBA3E0FAA3E0F92290010274B4
:10361C0001F09041267482F0A3F0A3F0A3F0E4A390
:10362C00F022EBF0A3EAF0A3E9F01213C4FD22742C
:10363C00C0F074A8A3F0A37401F022904145F07B74
:10364C00017A417926229000031213DDFD229000AD
:0A365C00010213DD9000020213DDED
:0B37FF0090620BEBF0A3EAF0A3E9F0EE
:10380A00E4A3F090620EE0FD2409FFE433FE906227
:10381A000B12360F8D827583001213DDFD123C11D7
:0C382A0090620EE004F0E0C3940640D76A
:01383600226F
:1038A60090620B12362E7F017E00123C1112360CEE
:1038B60012365AFD7F027E00123C1112360C123669
:1038C60060FD7F037E00123C1112360C1236527FC9
:0638D600047E00023C111B
:1037490090620B12362E7F057E00123C1190620B9F
:1037590012360F12365A7F0612377C12360F12367E
:10376900607F0712377C12360F1236527F087E00AF
:0D377900023C11FD7E00123C1190620B22FB
:1037860090620B12362E7F0F7E00123C1190620B58
:1037960012360F12365A7F101237B912360F1236FA
:1037A600607F111237B912360F1236527F127E0021
:0D37B600023C11FD7E00123C1190620B22BE
:103A2B00123618A3F090413212363BA374AEF0A3BA
:103A3B0074FF123625A312363B745E123640E41225
:0C3A4B003647123B5B9021047401F0220E
:10370300123618A3F0A3F0A37408F0A374DCF0A39B
:103713007411F0A37499F0A37477F0A3740AF0A35F
:103723007401F0A3F0A374FBF0A374FF123625A376
:10373300740AF0A37401123625123647123B5B90CC
:0637430021057401F022D3
:1035AE0012364B123C9D904126E0FFB48203308BC5
:1035BE00051237038024308905123A2B801C904166
:1035CE002AE0B40106A3E06425600F90412A74013D
:1035DE00F0A3742512364A123B5B7B017A41793295
:1035EE001237867B017A41793A1238A67B017A41ED
:0E35FE0079361237497B017A41792C0237FF6A
:103C3B00AE028EFB8FFAE4FBFDFC22EBF0A3EAF065
:053C4B00A3E9F0E422F2
:1039FE00E490620EF0A2AF33F0C2AF53FFBF8FF16F
:103A0E00AE04AF058EF38FF2AF038FF41207FD43B2
:0C3A1E00FF4090620EE024FF92AFAFF476
:013A2A002279
:103B5B0090620B123C46FBFDFC7FD01239FE90624B
:0F3B6B000BA3E0FAA3E0FF123C3B7FD10239FE2F
:0A3C9D00AF01123C3B7FD20239FE5A
:103AF200AC02AD018CFB8DFA9062A4E0FCA3E0293C
:103B0200F9EA3CAD01F5FD8DFCAD07AC06E4FB7FA7
:043B1200A10239FED5
:0934DE0090628FEEF0A3EFF0A361
:1034E700123C46906296F0A3F0906294E0FEA3E04F
:1034F700FFA3E0FCA3E0FDC39FEE6480F8EC6480CB
:10350700985041906290E02DFF90628FE03CCF246D
:10351700FFCF34FF8F82F583740193FF906291E0B0
:10352700FBA3E0FAA3E0F9906296A3E0F5828C830F
:10353700EF12141C906297E004F070AD906296E071
:0435470004F080A567
:01354B00225D
:10700000C2AF75FF407F717E001271D17F617E003B
:107010001271D1E4900000F0A3F0FFFE1271B77F6F
:10702000007E681271B753FFBF75F18012000A75B8
:10703000F130900000E0FEA3E0FF8EF38FF2E4F564
:10704000F412000A43FF401271AF53FFBF75F1A065
:10705000900000E0FEA3E0FF8EF38FF2E42FF582B4
:1070600074803EF583E0F5F412000A43FF4090007F
:1070700001E004F07006900000E004F0D3900001FD
:10708000E09400900000E0946840097F317E001297
:1070900071D1800C900000E05403FEA3E04E70AA72
:1070A000A2A2B392A2A2A3B392A3C3900000E094C1
:1070B0006850030270267F427E001271D1E4900076
:1070C00000F0A3F01271AFC20020003853FFBFE4FC
:1070D000F5F1900000E0FEA3E0FF8EF38FF21200C6
:1070E0000AAFF443FF40900000E0FCA3E0FDE42D74
:1070F000F58274803CF583E06F6009D2007F437EA7
:10710000001271D1900001E004F07006900000E0E0
:1071100004F0D3900001E09400900000E0946840F7
:10712000097F327E001271D1800C900000E0540380
:10713000FEA3E04E7093C200A2A2B392A2A2A4B397
:1071400092A4C3900000E0946850030270C4C2A2ED
:10715000D2A3D2A47F7A7E001271D1020000AD07C3
:10716000EDC4540FFFC3940A400BEF75F00A84E599
:10717000F02441800CEDC4540F75F00A84E5F0242E
:1071800030FFE433FE1271D1ED540FFFC3940A4077
:107190000BEF75F00A84E5F02441800BED540F7578
:1071A000F00A84E5F02430FFE433FE1271D122901E
:1071B0000000E0FEA3E0FFAB07AA06EAFF12715E43
:1071C000AF0312715E7F0D7E001271D17F0A0271D2
:0971D000D18F993099FDC299227A
:102E2B000D0A4143434553204554482D44494F2DEA
:102E3B0034382055706C6F616420506F727420436E
:102E4B006F6E6E65637465640D0A0055706C6F610F
:102E5B006420446174616772616D3A2025730D0AB9
:102E6B00005374617475733D382C206C696E656CFE
:102E7B00656E6774683D25303262782066756C6CC0
:102E8B00646174616772616D3D25303262782063D5
:102E9B006F6D706172653D253032627800537461DD
:102EAB007475733D31302C206C696E656373756D71
:102EBB003D2530326278206373756D5F63616C639F
:102ECB003D25303262782C2073756D3D2530326292
:102EDB0078200D0A006C61756E6368696E672066F9
:102EEB006C61736820636F7079206F7065726174A9
:102EFB00696F6E2066726F6D20253034780D0A0075
:102F0B000D0A666C61736820636F7079207265744B
:102F1B0075726E65643F213F21213F20756E657888
:102F2B007065637465642073686F756C6420686189
:102F3B00766520637261736865642E2E2E2E0D0AE2
:012F4B000085
:0C3B8A00414146004141470041414800D4
:101FF6002406F582E43EF583E0FD7F007E801238FC
:10200600609061FCE0FEA3E02407F582E43EF583E0
:10201600E0FD7F017E801238609061FCE0FEA3E067
:102026002408F582E43EF583E0FD7F027E801238C7
:10203600609061FCE0FEA3E02409F582E43EF583AE
:10204600E0FD7F037E801238609061FCE0FEA3E035
:10205600240AF582E43EF583E0FD7F047E80123893
:10206600609061FCE0FEA3E0240BF582E43EF5837C
:10207600E0FD7F057E80123860906202E0FBA3E0FF
:10208600FAA3E0F9740512140A906202E0FBA3E0D9
:10209600FAA3E022740490000512141C9061F9E082
:1020A6009061FCFFE0FCA3E090620FAA04F97B01BB
:1020B600E4F0A322906200E0FEA3E0FF240CFDE41E
:1020C6003EFC9061FCE0FAA3E0FB2DF582EA3CF5CC
:1020D60083E0F9906209F0EF2406FFE43EFEEB2F61
:1020E600F582EA3EF583E090620AF0FEE95E9062D0
:1020F60009F0EEF4A3F0229001027401F022F990A7
:1021060000051213DD904132F09000061213DD90A7
:102116004133F09000071213DD904134F09000082F
:102126000213DD9061F9E09061FCFFE0FCA3E0AAF8
:1021360004F97B01A3E0FDA3E090620FCDF0A3EDCF
:10214600F022FAA90790620C7401F0A3EAF0A3E961
:10215600F022F9E43AFA0D0239C0904150E090625B
:1021660000FFE0FCA3E0FDC39FEC221213C4FFFDB9
:102176003395E0FC906166E02DF0906165E03CF0FF
:1021860022F99000050213DDEEF0A3EFF0D39400E0
:10219600EE940022E0FFA3E0FAA3E0FB90620F7446
:1021A60020F07D0122E02430F0906165E03400F0FB
:1021B60022EFF0A3ECF0A3EDF0A3EAF0A3EBF0F925
:1021C60022F99000010214FAF09000060213DDF0E5
:1021D6009000070213DDC3906201E094069062004E
:1021E600E09400222DFD9061FCE03400FAA9057B05
:1021F60001229061FCE0FEA3E022906205E024004B
:10220600FFE43480FE22E4906200F0A3F022F09016
:1022160000090213DDF090000A0213DDF91213C45F
:10222600FFC3648094C122F582E43EF58322906266
:1022360001E004F022906200E004F022E0FF9061E9
:06224600FCE0FCA3E02215
:10383700F9906200E0FEA3E0FF240CF582E43EF578
:10384700831213DDFD90620AE05DFD906209E04D91
:09385700FDF0E42FFFEE3480FEC9
:043860008F828E8342
:0A386400AF05759301EFF0E4F59352
:01386E002237
:1039A100F9906200E0FEA3E0FF240CFDE43EFCE997
:0F39B1002DF9EA3CFAE42FFFEE3480FEAD07FC5F
:0439C0008D828C83E5
:0C39C400759301E0FFE4F593EF02140A94
:030800009061F90B
:100803001221B790620212214EE4906208F09061C7
:10081300F9E0FF123C26EF7003020D4F24ED700345
:10082300020D6024F77003020D4724056003020DD7
:0D083300689061F9E0FF123CA7EF30E0573C
:10084000E4906209F0906209E0FFC39407503E9083
:1008500061F9E0FEEF6E602D906209E0FF123C2628
:10086000BF1722E49061FEF0A3F0906209E0FF90D0
:1008700061FCE0FCA3E0AA04F97B01E490620FF0C4
:10088000A3F0122BC2906209E004F080B89061F9E5
:07089000E0FF7D01123C8531
:100897009061F9E0FF1236669061FE12218E5003D7
:1008A700020D689061F9E09061FC12213012331952
:1008B7009061FEEEF0A3EFF012208F1221C7121500
:1008C7006E0B53436847570AFD4368494F0B2C4348
:1008D7006849500C5643684D430BC543684E500B4F
:1008E700C543684E570B8C4368534D09FE44494F27
:1008F7002109805241444909325241574C0D275230
:100907005044490CA9525374610D07554461740D45
:100917000B5546696E0A195741444F0A3A575044D6
:100927004F0A775752504400000D27906208740110
:10093700F01221F8240612222DE0FF131313541F7F
:10094700FE906205F0EF5407A3F07B017A62790706
:10095700EE2400FFE41239BA122200906207E0FD8C
:10096700906206E0FC7401A804088002C333D8FC37
:100977006DFD906207F01238601220FD12208FF98A
:10098700740B12208CF990000112154A525F4F4BDD
:10099700900005740612141CE92406F9E43AFA7D5E
:1009A700007C801239C012208F2407122158122090
:1009B7008F240812215812208F240912215812203F
:1009C7008F240A12215812208F240B12215890626B
:1009D70008E0601B122200A3E0FD7401A80508804F
:1009E70002C333D8FCFD906207E06DFD1238601238
:1009F70020A2740C020D431220FD12207FF99000F3
:100A07000112154A5F457272743212209C740602F5
:100A17000D431220FD1221F8121FF6F99000011262
:100A2700154A575F4F4B900005740612209F7406B6
:090A3700020D431220FD12220CF5
:0F0A40001220BA12208F1239A112208F123837CC
:100A4F00122234700312223B1221DC40E412207F69
:100A5F00F990000112154A575F4F4B90000574062D
:0E0A6F0012209F7406020D431220FD12220C6D
:100A7D001220BA12208F1239A112208F123837127C
:100A8D00208FF9906200E0FEA3E0FF24061239AC3E
:100A9D00122234700312223B1221DC40D312208F1C
:100AAD001221C77B4F7A4479507857C31214D690D0
:100ABD006202701B122082F990000112154A575FD5
:100ACD004F4B900005740612209F7406020D4312C1
:100ADD002092F9741112208CF990000112154A52CE
:100AED005F4F4B900005740C12209F7412020D4342
:100AFD001220FDC2B61221F8FF240D12222DE05452
:100B0D003FF5B0EF121FF6F990000112154A575F2D
:100B1D004F4B900005740612209F7406020D431270
:100B2D0020FD12208F122104904135F012208AF9F8
:100B3D0090000112154A575F4F4B12209A120D6902
:100B4D00120D94020C531220FD12208F122187904A
:100B5D00413A1221CE90413B1221D590413C1221B8
:100B6D002290413DF012208AF990000112154A574A
:100B7D005F4F4B12209A120D69120D9E020C5312EB
:100B8D0020FD12208F1221879041361221CE9041E7
:100B9D00371221D5904138122122904139F012207F
:100BAD008AF990000112154A575F4F4B12209A1285
:100BBD000D78120DA8020CA01220FD12208F12210B
:100BCD000490413512221490413612221B90413768
:100BDD00F090000B1213DD904138F090000C1213C1
:100BED00DD904139F090000D1213DD90413AF090F7
:100BFD00000E1213DD90413BF090000F1213DD90AB
:100C0D00413CF09000101213DD90413DF012208A0E
:100C1D00F990000112154A575F4F4B12209A120D91
:100C2D007812208F1221C77B577A4E79687843C38B
:100C3D001214D6700B120D94120DA8120D9E800673
:100C4D009021037464F0020CA01220FD12208F126B
:100C5D00218790412C1221CE90412D1221D590410A
:100C6D002E12212290412F12221490413012221B5C
:100C7D00904131F012208AF990000112154A575F08
:100C8D004F4B12209A7406120D877B017A41792CF5
:100C9D001237FF7B017A417926023B5B1220FD1250
:100CAD00208FF9742412208CF990000112154A52EC
:100CBD005F4F4B12220C906200E0FEA3E0FF7B0120
:100CCD002426F974413EFA1213C4FD12208F240517
:100CDD00F9E43AFAE92FF9EA3EFAED12140A122272
:100CED0034700312223B906200E07004A3E0642094
:100CFD0070C41220A27425020D431220FD22122071
:100D0D00FD12207FF990000112154A575F4F4B904D
:100D1D000005E412209F7406801C1220FD12208F06
:100D2D00F9740412208CF990000112154A5F457276
:100D3D00721220A27405120D87229061F9E0FF0254
:100D4D003BB29061F9E0FF123B169061F912219AC6
:0B0D5D000232499061F9E0FF12386F8C
:100D6800227406F0122BC29061FEEEF0A3EFF0227F
:100D78007406F0122BC29061FEEEF0A3EFF022F0A1
:100D8800122BC29061FEEEF0A3EFF0227B017A41B4
:100D98007932123786227B017A41793A1238A622B3
:0A0DA8007B017A41793612374922A7
:10346900E490620CF0A3EB122150122171123AA7D9
:10347900501990620D1220921222225005EF24D089
:1034890080051213C424C990620CF090620EE47591
:10349900F00112143E90620D122092F912217190DE
:1034A900620CE0FEC454F0F0123AA7501C90620D71
:1034B9001220921222225005EF24D080051213C443
:1034C90024C9FF90620CE02FF090620CE0FF90613C
:0434D90069E02FF087
:0134DD0022CC
:10390F00906209EB1221509062091220922402F961
:10391F00E43AFA1234697E00C006C00790620912B9
:10392F002092F9123469EFFCD0E02400FFD0E03C84
:02393F00FE2266
:030DB2009061F954
:100DB5001221B790620212214EA312214EE4A3F034
:100DC5009061F9E0FF123C26EF700302127D24EDDD
:100DD500700302128E24F770030212572405600374
:100DE5000212969061F9E0FF123CA7EF30E01890EF
:100DF50061F9E0FF7D01123C85E4904146F07BFFFF
:100E05007A2E792B121A6C12129712219350030223
:100E15000EA9904146E070299061F9122242906234
:100E25000F1220B1041212A89061FCE0FEA3E0F5B8
:100E3500828E83E0904147F09041467401F0020EA6
:100E4500A9904147E0FFD39061FFE09F9061FEE0EC
:100E550094009061F9E0FF904146E0FD9061FDE06E
:100E650050101221EA9061FEE0FDA3E090620FCDE3
:100E7500800C1221EA904147E0FD90620FE4F0A357
:100E8500ED1212A89061FEA3E0FF904146E02FF01D
:100E9500A3E0C39FF0700D904146E0906208F0E436
:100EA500904146F0906208E0700302125190620290
:100EB5001220921221C712156E0F4F5544617411FD
:100EC500A85546696E0ED455706C64000012511217
:100ED50020FDE4904147F0A3F0A3F0906169F09004
:100EE5006165F0A3F090414EF0A3F0906163F0A32B
:100EF500F090414CF0A3F074FF90414AF0A3F090BC
:100F050041487401F0A31221CEFE1221887C0024F1
:100F150000FFEC3E90414EF0A3EF122122FE12217C
:100F2500D62400FFEC3E4F60069041497420F090B6
:100F35006202122092F912221CFE1222157C002454
:100F450000FFEC3E90616702124D1220FD90414872
:100F5500E064016003021251A3E0FF640160030233
:100F650011A0906205122092122187643A6008EF61
:100F75004402904149F022906166E0243A1221AE84
:100F850090000C12147F64307004E5F06430600842
:100F9500904149E04404F0229061661221ABA3120E
:100FA50021AB9062051220922406F9E43AFA123434
:100FB50069904150EFF09062051220922408F9E4FF
:100FC5003AFA12390F906161EEF0A3EFF0904150BB
:100FD500E0F92FFFE43ECF24FFCF34FFFEC390415D
:100FE5004DE09F90414CE09E5005EEF0A3EFF09050
:100FF500414AE0FEA3E09061611221679E5008908E
:10100500414AECF0A3EDF0906208E0FD24F0FBE42A
:1010150034FFFAE975F002A46B7003E5F06A603CF1
:10102500904149E04408F09061FCE0FEA3E0FF2D0B
:1010350012222DE4F0EF2405FFE43E12214812129E
:10104500C27A2E796C904150E025E090620CF090C8
:101055006208E090620DF024F0021110E490620045
:10106500F0A3F01221609400503E90620512209288
:10107500240EF9E43AFAED25E0FFEC33FEE92FF909
:10108500EA3EFA123469906200E0FCA3E02451F5CF
:101095008274613CF583EFF0906201E004F070C367
:1010A500906200E004F080BB906205122092240E4D
:1010B500F9E43AFA904150E075F002A429F9EA35CD
:1010C500F0FA12346990616AEFF0906169E060406E
:1010D500904149E04410F0906208122242FD2FF53C
:1010E50082E43CF583E4F0ED2405FFE43C1221485D
:1010F5001212C27A2E79A890616AE0FF90620CF014
:10110500906169E0FE90620DF0EF2EA3F0021A6C7B
:10111500906164E004F07006906163E004F0904132
:101125004EE0FEA3E0FF906163E0B5062AA3E0B5BB
:101135000725904149E054FEF0906165E0FEA3E08B
:10114500FF906168E02FFF906167E03E4F60089077
:101155004149E04440F022E4906200F0A3F01221FE
:10116500609400400302125174512DF58274613C64
:10117500F583E0FF906162E02DFD906161E03CFC4C
:10118500E42DF58274803CF583EFF0906201E00474
:10119500F070CB906200E004F080C3904149E044D8
:1011A50080F0221220FDE4904148F0A3E090620215
:1011B500704B122092F9740412140A9062021220E4
:1011C50092F990000112154A575F4F4B9061F9E073
:1011D5009061FC1220A974051212B5C2AF7BFF7A8B
:1011E5002E79E090620C7470F0A3E4F0121A6C1280
:1011F50070007BFF7A2F790B121A6C8034122092C3
:10120500F9740512140A906202122092F9900001F5
:1012150012154A5F457272904149E090000512141B
:101225001C9061F9E0FF9061FC1220AA740612126D
:10123500B5E4904146F0121297122193400E122107
:10124500291233199061FEEEF0A3EFF0E4906208E5
:10125500F0229061F9E0FF1236669061FE12218E50
:10126500400E1221291233199061FEEEF0A3EFF022
:101275009061F9E0FF023BB29061F9E0FF123B1685
:101285009061F912219A0232499061F9E0FF123812
:011295006FE9
:10129600229061F9E0FF1236669061FEEEF0A3EF50
:1012A600F022F01233199061FEEEF0A3EFF022F077
:1012B600122BC29061FEEEF0A3EFF0227BFF7A2E96
:0812C6007956121A6C7BFF221D
:030000000233DDEB
:0C33DD00787FE4F6D8FD758121023424CD
:1012CE00E709F608DFFA8046E709F208DFFA803E02
:1012DE0088828C83E709F0A3DFFA8032E309F608EF
:1012EE00DFFA8078E309F208DFFA807088828C8357
:1012FE00E309F0A3DFFA806489828A83E0A3F6080B
:10130E00DFFA805889828A83E0A3F208DFFA804CE4
:10131E0080D280FA80C680D4806980F280338010BB
:10132E0080A680EA809A80A880DA80E280CA803324
:10133E0089828A83ECFAE493A3C8C582C8CCC5839C
:10134E00CCF0A3C8C582C8CCC583CCDFE9DEE7806C
:10135E000D89828A83E493A3F608DFF9ECFAA9F0EB
:10136E00EDFB2289828A83ECFAE0A3C8C582C8CC41
:10137E00C583CCF0A3C8C582C8CCC583CCDFEADE5A
:10138E00E880DB89828A83E493A3F208DFF980CCBC
:10139E0088F0EF60010E4E60C388F0ED2402B404B5
:1013AE000050B9F582EB2402B4040050AF2323455C
:0613BE00822390131E7350
:1013C400BB010689828A83E0225002E722BBFE0227
:0913D400E32289828A83E493225A
:1013DD00BB010CE58229F582E5833AF583E02250C5
:1013ED0006E92582F8E622BBFE06E92582F8E2220F
:0D13FD00E58229F582E5833AF583E4932229
:10140A00BB010689828A83F0225002F722BBFE01C1
:02141A00F322BB
:10141C00F8BB010DE58229F582E5833AF583E8F006
:10142C00225006E92582C8F622BBFE05E92582C8B2
:02143C00F2229A
:10143E00C5F0F8A3E028F0C5F0F8E5821582700239
:06144E001583E038F022D6
:10145400BB010A89828A83E0F5F0A3E02250068763
:10146400F009E71922BBFE07E3F5F009E319228925
:0B147400828A83E493F5F07401932258
:10147F00BB0110E58229F582E5833AF583E0F5F0AB
:10148F00A3E0225009E92582F886F008E622BBFE88
:10149F000AE92582F8E2F5F008E222E5832AF583CE
:0814AF00E993F5F0A3E9932293
:1014B700BB010A89828A83F0E5F0A3F0225006F780
:0F14C70009A7F01922BBFE06F3E5F009F319227D
:1014D600EB9FF5F0EA9E42F0E99D42F0E89C45F06C
:0114E60022E3
:1014E700E8600FECC313FCED13FDEE13FEEF13FFE3
:0314F700D8F12207
:1014FA00BB010DE58229F582E5833AF5830215B42D
:10150A005007E92582F80215A8BBFE07E92582F8EB
:10151A000215C0E58229F582E5833AF5830215CCE6
:10152A007401FF3395E0FEFDFC080808E6CF2FF6AC
:10153A0018E6CE3EF618E6CD3DF618E6CC3CF62285
:10154A00BB010DE58229F582E5833AF5830215F59B
:10155A005007E92582F80215DCBBFE07E92582F867
:04156A00021626221D
:10156E00D083D082E4937012740193700DA3A39371
:10157E00F8740193F5828883E4737402936C70128D
:10158E007403936D700C7404936E70067405936FF0
:0A159E0060DDA3A3A3A3A3A380CAEA
:101A0100E508240CF582E43462F583E005082290B0
:101A1100620930070390620CE475F00112163F026F
:101A210013C42000E97F2ED2008018EF540F2490B8
:101A3100D43440D4FF30040BEF24BFB41A00500358
:101A41002461FFE50960021509050CE50C7002052A
:101A51000B30070E906209E475F00112163FEF0298
:101A6100140A023CB07403D2078003E4C207F508EC
:101A7100906209121656E4F509F50BF50CE50960BB
:101A8100077F20121A4480F5750AFFC201C200C205
:101A910002C203C205C206C208121A10FF700D303D
:101AA10007057F00121A55AF0CAE0B22B4255FC299
:101AB100D5C204121A10FF24D0B40A00501A75F0CE
:101AC1000A780930D50508B6FF0106C6A426F62016
:101AD100D5047002D20380D924CFB41A00EF500488
:101AE100C2E5D204021C56D20180C6D20080C0D207
:101AF1000280BCD2D580BAD20580B47F20121A44AC
:101B01002002077401B5090040F1121A01FF121AEF
:101B110044021A7ED208D2068095121A01FB121ACB
:101B210001FA121A01F94A4B700679277A1D7BFFD7
:101B310020022EE509602A7E008E82758300121331
:101B4100DD60060EEE650A70F0C2D5EBC0E0EAC0BA
:101B5100E0E9C0E0EE121C9DD0E0F9D0E0FAD0E05F
:101B6100FB1213C4FF60AAEBC0E0EAC0E0E9C0E0E9
:101B7100121A44D0E02401F9D0E03400FAD0E0FB9D
:101B8100E50A0460DCD50AD980877BFF7A1C799944
:101B9100D202809C791080027908C206C2088008AE
:101BA100D2D5790A8004790AC2D5E50A047002F512
:101BB1000AE4FAFDFEFF121A01FC7B082001131250
:101BC1001A01FD7B1030000A121A01FE121A01FFE0
:101BD1007B20EC3382D592D55013C3E43000069FAD
:101BE100FFE49EFEE42001039DFDE49CFCE4CBF8B0
:101BF100C201EC700CCFCECDCCE824F8F870F380A4
:101C010017C3EF33FFEE33FEED33FDEC33FCEB3363
:101C1100FB994002FB0FD8E9EB300105F8D0E0C495
:101C210048B201C0E00AEC4D4E4F78207B0070C2F3
:101C3100EAB50A0040BCC0E0121C9FD0F0D0E02001
:101C41000104C4C0E0C4B201C0F0121A2DD0F0D515
:101C5100F0EB021A7E12165F1B1B531B95581AECF0
:101C61004C1AE8421B994F1BA1441BA1491B01437C
:081C71001BA7551B8B461B8BC2
:101C7900451B8B471D47501AF02D1AF42E1B172BA5
:101C89001AF8231B15201D302A1AB04800001B0F13
:101C99003F3F3F00790AA2D5200314300509B91046
:101CA900020404B9080104A2D52006025001042047
:101CB90002689202B509005034C0E07F2030031950
:101CC9007F30A20272067205500F121CF6C202C2C0
:101CD90006C205C2087F30800F300503E9C0E01253
:101CE9001A44300503D0E0F9D0E0B509CC30051726
:101CF9007F30B9100C121A447F583004077F78805E
:101D090003B90803121A443002057F2D021A447FD1
:101D1900202008F87F2B2006F322920280CF286E1C
:101D2900756C6C2900D201121A013001F8C20178D0
:101D39000930D50108F6021AB02D50434958121A34
:101D4900012403B405004001E4901D4293121A35A1
:0D1D5900743A121A35D203750904021B9565
:103AA700EFC394414005EF94474016EFC39461403C
:103AB70005EF9467400BEFC394304008EF943A50FA
:063AC70003D38001C322BD
:1033E900021685E493A3F8E493A34003F68001F25F
:1033F90008DFF48029E493A3F85407240CC8C333E5
:10340900C4540F4420C8834004F456800146F6DFB3
:10341900E4800B0102040810204080903B7AE47E8E
:10342900019360BCA3FF543F30E509541FFEE493A8
:10343900A360010ECF54C025E060A840B8E493A36F
:10344900FAE493A3F8E493A3C8C582C8CAC583CA9A
:10345900F0A3C8C582C8CAC583CADFE9DEE780BE52
:013B9600002E
:0C15A800E6FC08E6FD08E6FE08E6FF226F
:0C15B400E0FCA3E0FDA3E0FEA3E0FF22AA
:0C15C000E2FC08E2FD08E2FE08E2FF2267
:1015CC00E493FC740193FD740293FE740393FF2265
:1015DC00D083D082E493F608740193F608740293D6
:0915EC00F608740393F67404730D
:1015F500A8828583F0D083D08212160C12160C12A5
:10160500160C12160CE473E493A3C583C5F0C583C9
:10161500C8C582C8F0A3C583C5F0C583C8C582C83F
:0116250022A2
:10162600D083D082E493F208740193F20874029393
:09163600F208740393F2740473CA
:10163F00F8E0FBA3A3E0F925F0F0E5821582700234
:07164F001583E0FA38F022D8
:09165600EBF0A3EAF0A3E9F02295
:10165F00D083D082F8E4937012740193700DA3A31A
:10166F0093F8740193F5828883E47374029368602E
:06167F00EFA3A3A380DF2E
:00000001FF
